:100000000C94EE010C9426020C9426020C94260209
:100010000C9426020C9426020C9426020C942602C0
:100020000C9426020C9426020C94471B0C94191C69
:100030000C9444160C9426020C9426020C9426026E
:100040000C9426020C9426020C9426020C94260290
:100050000C9426020C94CC160C9426020C942602C6
:100060000C9426020C9426020C9426020C94260270
:100070000C9426020C9426020C9426020C94260260
:100080000C9426020C9426020C9426020C94260250
:100090000C9426020C9426020C9426020C94260240
:1000A0000C9426020C9426020C942602DA04DA043C
:1000B000060506056E059906990699068C0525061E
:1000C00036063606861CAD1CA51DAD1CA51DF91CEB
:1000D0001C1DA51D731D821D4C00E000490042003F
:1000E0002D0041002E002300000022004A003B00AA
:1000F0004B003A00350000004800000000001300EB
:1001000012000C0018004700150000000800000055
:100110001A00140000003E000000430027002600E3
:1001200025002400460021004D0020004E001F0045
:100130001E002C00000000004400340000003F00BE
:100140000B00E2000A0052003D0000000000290000
:100150000000000000002A002F00400030001C00BA
:1001600000001700E3003C00E10039002B00000014
:10017000E4000000280000003700360010000000F6
:1001800019000000060000001B001D0051000000C7
:100190004F0045003800015100001100E600050045
:1001A000500000000000000000000000E700000018
:1001B000310033000F000E000D00000009000000A8
:1001C0000700E50016000400AC000100AE000100CD
:1001D000010001000100010000000100AD0001006C
:1001E000A900010001000000A800000000000100BB
:1001F00001000100010001000100000001000000F9
:1002000001000100000001000000010001000100E8
:100210000100010001000100AB000100AA00010083
:100220000100010000000000C15C010000000100AD
:100230000100010001000100010000000000005C5D
:1002400000000000000001000100010001000100A9
:100250000000010001000100010001000100000098
:100260000100000001000000010001000100000089
:100270000100000001000000010001000100000079
:100280000100C05C0100010000000100010001004C
:10029000010000000000000000000000010000005C
:1002A0000100010001000100010000000100000048
:1002B00001000100010001001403510075006100FC
:1002C00063006B00660069007200650000000E03A9
:1002D000450076007900640031003300000004031B
:1002E000090409023B00020100A0FA090400000110
:1002F00003010100092111010001224000070581CD
:100300000308000109040100010300000009211194
:10031000010001226D000705820320000112010087
:1003200002000000080547C987010001020001051D
:10033000010980A101850319012AB700150126B71B
:1003400000950175108100C0050C0901A10185040B
:1003500019012AA002150126A0029501751081003D
:10036000C005010906A1018506050719E029E71561
:100370000025019508750181020507190029EF156F
:1003800000250195F07501810205081901290595DF
:100390000575019102950175039101C005010906DA
:1003A000A101050719E029E7150025019508750148
:1003B00081029501750881010507190029FF1500C3
:1003C00026FF009506750881000508190129059585
:1003D0000575019102950175039101C011241FBE9D
:1003E000CFEFDAE0DEBFCDBF04B603FE18C08091C8
:1003F000DD029091DE02A091DF02B091E002873031
:10040000904BA740B04B59F41092DD021092DE02DF
:100410001092DF021092E002E0E0F8E3099511E0AB
:10042000A0E0B1E0E0E6FCE302C005900D92AA383E
:10043000B107D9F722E0AAE8B1E001C01D92AD3DB5
:10044000B207E1F70E94A4120C942E1E0C94000037
:1004500081E0089581E008950C942A0208950C9497
:100460002E021F93CF93DF9300D000D01F92CDB701
:10047000DEB749835A836B8330918D0189819A81DC
:10048000311114C0662359F0222349F00E94D2088A
:10049000182F682F89819A810E947B0803C00E94CF
:1004A000A608182F69817A81812F04C00E94D20882
:1004B00069817A810F900F900F900F900F90DF91CC
:1004C000CF911F910C94F60FFC01262F4081518192
:1004D0006281738184810C94310281E00895CF930D
:1004E000DF93EC0160E00E946402BE01DF91CF91D6
:1004F0000C942F020C943C110C94381108950E9416
:1005000025070E947E022FEF84E39CE0215080406B
:100510009040E1F700C000000C94F2160F931F9377
:10052000CF93DF938C0161E00E946402EC01B8017B
:100530000E942C028823F1F1B801CE010E949D1483
:100540008823C1F1B801CE010E94B112882391F134
:10055000B801CE010E94F913882361F1F80182816C
:10056000882309F1CB358DE5D807C1F050F4C115CA
:10057000FCE5DF0781F0CF3DDC45A9F40E94090EC0
:1005800019C0CC35EDE5DE0761F0CD35DD4559F418
:100590000E944C0D08C00E947F020CC00E94550DA5
:1005A00002C00E94580DC801DF91CF911F910F9199
:1005B0000C94280280E0DF91CF911F910F91089554
:1005C0000E9426160C940E030E9411030C942C1604
:1005D00008950C94E80281E00895CF93C82F0E94FB
:1005E000EB02882359F0C095C1FF02C08F9A01C069
:1005F0008F98C2FF02C08E9A01C08E98CF91089545
:10060000879A8F9A869A8E9A0895CF93C82F0E94C0
:10061000E9028C2F0E94ED02CF91089580E00C94A6
:1006200005030E94F9140C9405030E94F91490919B
:100630008C01891721F080938C010C940503089597
:10064000CF93DF93CDB7DEB72B970FB6F894DEBF0D
:100650000FBECDBF4F83588769877A878B8761111B
:100660000E94980C9E012F5F3F4F86E0F901119286
:100670008A95E9F785E0FE013796D90101900D9240
:100680008A95E1F789819A814C815D81452B31F012
:100690009F3F31F491E08F3F19F403C091E001C016
:1006A00090E090FF09C049815A816B817C818D81E6
:1006B0009E810E94B90B05C0C9010E946D02811183
:1006C000F2CF2B960FB6F894DEBF0FBECDBFDF91F1
:1006D000CF910895FC01808191810E9414090895B1
:1006E000CF93882309F49CC0C82F8238C1F40E949C
:1006F000F91481FD95C069E3809102019091030195
:100700000E94E1150E94BA0C2FEF81EE94E0215077
:1007100080409040E1F700C0000069E319C08338D1
:1007200001F50E94F91480FD7BC063E58091020110
:10073000909103010E94E1150E94BA0C2FEF81EE07
:1007400094E0215080409040E1F700C0000063E554
:1007500080910201909103010E94EC15CF910C94BD
:10076000BA0C8438C1F40E94F91482FD59C067E4C0
:1007700080910201909103010E94E1150E94BA0C40
:100780002FEF81EE94E0215080409040E1F700C0CF
:10079000000067E4DDCF8CEF8C0F813AD0F46C2F32
:1007A00080910201909103010E946115882349F014
:1007B0006C2F80910201909103010E94EC150E9420
:1007C000BA0C6C2F80910201909103010E94E115F7
:1007D000C5CF80E28C0F883048F4C77081E001C03B
:1007E000880FCA95EAF70E947B0CB8CFEBE5EC0FB7
:1007F000E33040F4F0E0E15CFE4F808190E0CF9187
:100800000C941F15C85AC73158F4EC2FF0E0EE0FC6
:10081000FF1FEF5EFE4F80819181CF910C943515C3
:10082000CF910895882309F45BC0682F823879F44A
:100830000E94F91481FF54C069E3809102019091F4
:1008400003010E94E1150E94BA0C69E310C08338CD
:10085000B1F40E94F91480FF43C063E58091020166
:10086000909103010E94E1150E94BA0C63E580910A
:100870000201909103010E94EC150C94BA0C84388B
:1008800079F40E94F91482FF2BC067E48091020181
:10089000909103010E94E1150E94BA0C67E4E7CF32
:1008A0008CEF860F813A18F380E2860F883048F487
:1008B000677081E001C0880F6A95EAF70E94810C99
:1008C000DCCF8BE5860F833020F480E090E00C9441
:1008D0001F15685A673120F480E090E00C943515BC
:1008E00008951F93CF93DF93182FEB010E9470039D
:1008F000209741F08FE99FE00197F1F700C00000D9
:100900002197F6CF812FDF91CF911F910C94120484
:10091000893319F060E070E002C060E570E00C948B
:100920007104882321F00E947B0C0C94BA0C08956A
:10093000882321F00E94810C0C94BA0C0895CF9268
:10094000DF92EF92FF920F931F93CF93DF937C017F
:10095000D62FC72FFC011281058102950F700E94CE
:10096000710C8823B9F01123A9F08C2F807F80347B
:1009700021F080E28D0F883068F08091AB0282FD1B
:1009800009C082E00E941A0D0E94710C91E0D82EDD
:10099000D92601C0D12CCC2EC2948FE0C8228C2D38
:1009A00090E08C30910508F0C4C1FC01EA5AFF4F79
:1009B0000C94D91D8C2F807FCF70882311F0C295A5
:1009C000C07F112399F0CC2309F49FC180E28D0FE1
:1009D000883010F0D11104C08C2F0E947B0C03C012
:1009E0008C2F0E948B0C0E94BA0C8FC18D2F0E94FD
:1009F0001204CC2309F49DC180E28D0F883038F1B8
:100A0000DD2329F18C2F0E94910C24C08C2F807F34
:100A1000CF70803211F0C295C07FDD2319F0D13044
:100A2000A1F13DC08091AB0282FF17C0112349F0B4
:100A3000CC2329F08C2F0E947B0C0E94BA0C80E002
:100A400065C180E00E941204CC2309F472C18C2F8E
:100A50000E94810C0E94BA0C6CC1112371F000231A
:100A600041F0013031F40E949B0C8C2B0E94A30CAE
:100A700060C10E949B0C8C2B1DC0002319F001301B
:100A800009F457C10E94B00C25C0112321F0063093
:100A900008F04FC10EC0053008F04BC11BC0112338
:100AA00061F0002331F0F701858180FF2EC18F7046
:100AB00085838C2F0E9491043CC1002359F0D933C7
:100AC00009F034C1FFEF07EE13E0F1500040104091
:100AD000E1F72AC18C2F0E9498042BC18C2F869598
:100AE0008695837019F0813061F023C1112321F0C4
:100AF0008D2F9C2F937002C080E090E00E941F1504
:100B000020C1112321F08D2F9C2F937002C080E013
:100B100090E00E94351515C18C2F837009F047C0F5
:100B200011110BC12D2F229526952770220F220F10
:100B30006D2F6F70862F90E0A0E0B0E0022E04C011
:100B4000880F991FAA1FBB1F0A94D2F7D4FF10C0A9
:100B50004FE050E060E070E004C0440F551F661F96
:100B6000771F2A95D2F7409550956095709503C0F0
:100B700040E050E0BA01C695C695C3708A019B015A
:100B8000082B192B2A2B3B2BC901B801C23049F085
:100B900058F4C13019F00E949107CFC00E947F071E
:100BA000CCC00E94A307C9C00E947D07C6C0112304
:100BB00019F08C2F817001C08695882309F4BDC07F
:100BC0002D2F229526952770220F220F6D2F6F70E3
:100BD000862F90E0A0E0B0E0022E04C0880F991F9D
:100BE000AA1FBB1F0A94D2F7D4FF10C04FE050E0F9
:100BF00060E070E004C0440F551F661F771F2A9500
:100C0000D2F7409550956095709503C040E050E054
:100C1000BA01C695C695C3708A019B01082B192B92
:100C20002A2B3B2BC901B801C23049F058F4C1301E
:100C300019F00E94560881C00E9444087EC00E949C
:100C400068087BC00E94B70778C0CF70112339F0C5
:100C50008C2F0E94DD078D2F0E9491046EC08D2F76
:100C60000E9498048C2F0E94FE0767C0D23F21F19A
:100C700028F4D03F41F0D13FC1F043C0D33F19F138
:100C8000D43F79F03EC0112341F0053008F051C047
:100C90008C2F8F710E9423084CC0063008F049C089
:100CA000F7CF8091AB0282FF18C0112339F08C2F4F
:100CB0008F710E94DD073DC01123C9F38C2F8F7106
:100CC0000E94FE0736C0112329F08C2F8F710E94DD
:100CD000C8072FC00E94C3072CC0112349F0CF7151
:100CE0008C2F0E94DD0763E08C2F0E94FF0C21C037
:100CF00081E00E941A0D0230E0F082E00E941A0D9D
:100D000018C0112331F0002391F28D2F0E9470033F
:100D100010C0002399F2D93349F41FEF27EE33E0D6
:100D2000115020403040E1F700C000008D2F0E949C
:100D3000120488EF8C0D843020F40E94F9140E9474
:100D40000503DD20C9F00E946D0C80FD15C0F70180
:100D500012820E94670C0E94DD07C7010E94DD0617
:100D60000E94670CDF91CF911F910F91FF90EF9040
:100D7000DF90CF900C94FE07DF91CF911F910F91E0
:100D8000FF90EF90DF90CF9008950F931F93CF9334
:100D9000DF93EC01688179818A810E941F098C01AF
:100DA0000E947A080E946B07B801CE010E949F043E
:100DB000DF91CF911F910F910895CF93DF93EC01B5
:100DC000988189812B813C81232B31F08F3F31F435
:100DD00081E09F3F19F403C081E001C080E080FD05
:100DE0001DC0CE010E948E02811110C00E94710CA4
:100DF0008823A1F08A81882389F08091AB0282FD4B
:100E00000DC082E0DF91CF910C941A0DCE010E94AB
:100E1000C506CE01DF91CF910C946F02DF91CF9187
:100E2000089580E090E00E941F1580E090E00E940D
:100E300035150E94980C0C94BA0C80910201909187
:100E400003010E94F7150C9411070E94880C0C9462
:100E50001D0792959F70963079F010F4925001C062
:100E60009A50923068F4803F69F018F4883E40F45C
:100E700009C0843F29F406C0883E20F0813F11F06C
:100E800080E0089581E00895FC01808191810E94B5
:100E900014090E9429070895CF93DF9300D000D052
:100EA0001F92CDB7DEB70F900F900F900F900F905D
:100EB000DF91CF910895CF93DF9300D000D000D081
:100EC000CDB7DEB726960FB6F894DEBF0FBECDBF06
:100ED000DF91CF910895089508950C946C070C94B8
:100EE0006D070E946F076093DD017093DE018093B0
:100EF000DF019093E0010C9411070C9471070F939C
:100F00001F930091DD011091DE012091DF013091EE
:100F1000E001602B712B822B932B1F910F910C946E
:100F200071070F931F930091DD011091DE01209155
:100F3000DF013091E00160237123822393231F910D
:100F40000F910C9471070F931F930091DD01109185
:100F5000DE012091DF013091E001602771278227B7
:100F600093271F910F910C9471070C946C070E94AA
:100F7000B5076093D9017093DA018093DB019093F8
:100F8000DC010C94110760E070E0CB010C94B70712
:100F90000F931F9341E050E060E070E08A019B01F5
:100FA00004C0000F111F221F331F8A95D2F7C901F9
:100FB000B8011F910F910C94B7070F931F9341E055
:100FC00050E060E070E004C0440F551F661F771FBB
:100FD0008A95D2F78091D9019091DA01A091DB0135
:100FE000B091DC018A019B01082B192B2A2B3B2B8A
:100FF000C901B8011F910F910C94B7070F931F936C
:1010000041E050E060E070E004C0440F551F661FEF
:10101000771F8A95D2F7409550956095709580918D
:10102000D9019091DA01A091DB01B091DC018A0134
:101030009B01082319232A233B23C901B8011F91CF
:101040000F910C94B7070F931F9341E050E060E0BD
:1010500070E004C0440F551F661F771F8A95D2F7B2
:101060008091D9019091DA01A091DB01B091DC016E
:101070008A019B01082719272A273B27C901B801A4
:101080001F910F910C94B7070F931F930091D901F3
:101090001091DA012091DB013091DC01602B712B82
:1010A000822B932B1F910F910C94B7070F931F93D3
:1010B0000091D9011091DA012091DB013091DC011E
:1010C00060237123822393231F910F910C94B70700
:1010D0000F931F930091D9011091DA012091DB0148
:1010E0003091DC0160277127822793271F910F9190
:1010F0000C94B70708952FE0929F800D1124E82FDC
:10110000E695E695E695877051E001C0550F8A9502
:10111000EAF785E0E89FF0011124E257FE4F20E056
:1011200030E070E04081CB01022E02C09695879599
:101130000A94E2F78170819584278523842781931F
:101140002F5F3F4F2530310569F708952FE0929FBB
:10115000800D1124682F669566956695982F977077
:1011600085E0689FB001112440E050E080E0FB0181
:10117000E40FF51FE257FE4F208130E0092E02C038
:10118000369527950A94E2F721703327042E01C083
:10119000220F0A94EAF7822B4F5F5F4F45305105CB
:1011A00031F70895BF92CF92DF92EF92FF920F93A3
:1011B0001F93CF93DF938C01C090D901D090DA01B7
:1011C000E090DB01F090DC018091DD019091DE0187
:1011D000A091DF01B091E001C82AD92AEA2AFB2AAE
:1011E000CFE1D0E0D701C6010C2E04C0B695A7957B
:1011F000979587950A94D2F780FD04C0219790F7C0
:10120000B12C07C0BC2EB8018C2F0E940910019789
:10121000A9F38B2DDF91CF911F910F91FF90EF904C
:10122000DF90CF90BF900895CF93DF93EC010E94A1
:10123000D208BE010E940910DF91CF9108951F933B
:10124000CF93DF93EB0190918D01992321F0CB0196
:101250000E94140913C0882349F0CB010E94D208D0
:10126000182F682FCE010E947B0804C0CB010E947A
:10127000A608182FBE01812F0E940910DF91CF917F
:101280001F9108951F93CF93DF93C091E10116E062
:101290008091E201C81799F0D0E01C9FF0011D9FDA
:1012A000F00D1124ED51FE4F408151816281738117
:1012B000848195810E945B072196C770E9CFDF91F9
:1012C000CF911F91089540911302509114026091A3
:1012D00015027091160280911702909118020C94D9
:1012E0005B07EF92FF920F931F93CF93DF93809151
:1012F000180282958F7009F065C0809115028823CD
:1013000009F460C08091E101F090E20110911302B4
:1013100000911402609116027091170291E01F3F34
:1013200009F090E0C0910001D0910101292F96E0D1
:10133000E92E8F1509F446C06115710521F00F3FA4
:1013400021F030E003C031E001C0322F90E030FDE9
:1013500036C0E89EF001E99EF00D1124DF01AD5189
:10136000BE4F11963C911197301329C03C91311317
:1013700026C012963C911297311121C013964D91BF
:101380005C911497461B570B4C175D07C0F4809176
:1013900018028F70806180931802E851FE4F80819F
:1013A0008F708061808383E192E00E94DD06DF918F
:1013B000CF911F910F91FF90EF900C9442090196ED
:1013C0008770B7CFDF91CF911F910F91FF90EF9072
:1013D00008959F92AF92BF92CF92DF92EF92FF92C9
:1013E0000F931F93CF93DF93CDB7DEB761970FB6FF
:1013F000F894DEBF0FBECDBF8C0185E0F801DE01A1
:101400001D9601900D928A95E1F7D8011296EC9005
:1014100090911302E091140220911602309117026C
:101420002115310531F0EF3F31F481E09F3F19F490
:1014300003C081E001C080E0B82FB1709B2E80FD19
:1014400047C1D8014C9111965C9111971396AD90BC
:10145000BC90149783E1C82E82E0D82EF09015023C
:10146000B501621B730B2091000130910101FF2037
:1014700009F4D9C0809118026217730708F095C06B
:10148000282F207F09F052C05E1313C0491311C0EA
:10149000FE2CE1100EC08F708061809318020E94B4
:1014A0006309C6010E94DD0680911802F801858358
:1014B0004DC1AB2831F05F3F31F481E04F3F19F46B
:1014C00003C081E001C080E080FD03C081E08E2583
:1014D00002C080E090E0F82FF170FF2E80FF1CC06A
:1014E0008091E1012091E20136E0821709F40BC1FD
:1014F00090E0389FF001399FF00D1124ED51FE4F1F
:101500006181561306C06081461303C06281E612F2
:1015100003C001968770E9CFFE2CEE2009F416C1B6
:101520008091180281608093180254C05E1306C037
:10153000491304C0E11002C0F80199C0C8010E941B
:101540004407882361F1EE2051F120911802822F87
:1015500082958F7090E0029774F0809113029091C1
:10156000140298878F831986BB86AA862C87CE01A2
:1015700007960E94DD0686E0F801A3E1B2E0019043
:101580000D928A95E1F70E9471090E9463090AC0D1
:101590005E1711F1C8010E94440781112CC0C801D7
:1015A0000E94DD06FF24F394D1C0282F207F81F70D
:1015B0007A2DB98AA88A6E2D89890E944C0783E109
:1015C00092E00E94DD0686E0D6011D928A95E9F739
:1015D0000E946309F12CBAC04913DCCFE110DACFC5
:1015E000F8018583C8010E94DD0686E0D6011D92C0
:1015F0008A95E9F7ABC0EE2091F220911802822F74
:1016000082958F7090E002970CF4B5CF8091130211
:10161000909114029A8389831B82BD82AC822E83AF
:10162000CE010196A6CF6217730708F044C0FE2CC6
:10163000EE2009F4B4CF5E1330C049132EC02091C0
:10164000180220FD21C0822F82958F70482F50E014
:1016500041155105C9F0F80125834F30510541F07E
:101660008F5F982F9295907F822F8F70892B858323
:10167000C8010E94DD0686E0F801A3E1B2E0019016
:101680000D928A95E1F73CC086E0F801A3E1B2E053
:1016900001900D928A95E1F759C0C8010E94440754
:1016A000811169CF80911802816080931802C8016E
:1016B0000E94DD064BC07A2DB98AA88A6E2D8989D1
:1016C0000E944C0786E0D6011D928A95E9F718C062
:1016D000EE2009F464CFC8010E944407F82E882345
:1016E00009F45DCF86E0F801A3E1B2E001900D922C
:1016F0008A95E1F783E192E00E946A030E947109F2
:101700000E94630923C04D875E878D859E850E9458
:101710001409292F22952F70223028F49F7039F058
:10172000811105C00BC0243028F49F7049F4805EFD
:10173000883020F0C8010E94DD069F2CF92C06C0DD
:10174000D80115969C91907F91F7F8CF8F2D6196D7
:101750000FB6F894DEBF0FBECDBFDF91CF911F91C2
:101760000F91FF90EF90DF90CF90BF90AF909F9040
:1017700008951F93CF93DF93CDB7DEB72C970FB6A5
:10178000F894DEBF0FBECDBF4F83588769877A8735
:101790008B879C87CE0107960E94E9098823D1F0A8
:1017A0009F8188852A853B85232B31F08F3F31F43B
:1017B00081E09F3F19F403C081E001C080E080FD1B
:1017C00047C04F81588569857A858B859C850E94A5
:1017D0005B073EC086E0FE013796DE011196019060
:1017E0000D928A95E1F7FF81E8856A857B85611511
:1017F000710531F0EF3F31F481E0FF3F19F403C090
:1018000081E001C080E080FD23C02091E20130E052
:10181000C9010196877099274091E10150E0841732
:101820009507F1F1F983EA837D836C8396E0929FBB
:10183000D001939FB00D1124AD51BE4FFE013196E2
:1018400001900D929A95E1F78093E2010E9442097E
:1018500016E08091E1019091E201891771F1189FE2
:10186000C00111248D519E4F0E94E909882329F15E
:10187000E091E1011E9FF0011124ED51FE4F4081E6
:10188000518162817381848195810E945B0780917F
:10189000E10190E00196877099278093E101D9CF0B
:1018A0000E9425071092E2011092E101E3E1F2E0CB
:1018B00086E0DF011D928A95E9F72C960FB6F89421
:1018C000DEBF0FBECDBFDF91CF911F9108958091F4
:1018D000390285958595859508958091390287709F
:1018E000089590913902977081E009F480E008959D
:1018F00080915C02089590915C02892B80935C0238
:101900000895809590915C02892380935C020895EC
:1019100010925C02089590915B02892B80935B0288
:101920000895809590915B02892380935B020895CE
:1019300010925B02089580913A02089508950C94E4
:101940009E0C0C949F0C9091AB0292FD08C090915C
:101950003A02981721F080933A020C94A10C089552
:1019600080913A02882329F010923A0280E00C9488
:10197000A10C0895CF93DF93E0910201F091030150
:1019800080915C028083E0910201F09103019081DB
:1019900080915B02892B808380913A02882381F0B9
:1019A000E0910201F09103019081892B8083809165
:1019B0000201909103010E944B1581110E94B00C0D
:1019C000C0910201D091030140E250E069E172E070
:1019D000CE010E94DF1D892B69F080E2FE01A9E1A2
:1019E000B2E001900D928A95E1F7CE01DF91CF919F
:1019F0000C940515DF91CF9108950C949E0C909155
:101A0000AB0292FD10C098E0899F90011124262B13
:101A1000209339020E94DD078091390285958595D2
:101A200085950C94FD0C0C94DD071092390280E032
:101A30000C94FD0C20913902809582238093390209
:101A4000982F977099F430E0482F082E000C550B12
:101A50002417350759F09091AB0292FD07C0859588
:101A6000859585950E94FE070C94150D089590911B
:101A7000AB0292FB222720F9281769F080FB92F92C
:101A80009093AB028091AA029091AB020E94850DC7
:101A900082E00C941A0D08958091AB0282FB882796
:101AA00080F991E089270C94370D81E00C94370D73
:101AB00080E00C94370D6FEF7FEF80E090E00C94A6
:101AC000181E80E090E00E94F41D21E0893E9E4FA8
:101AD00009F020E0822F089582E090E00C94EC1D44
:101AE00083E090E00C94EC1DCF9384E090E00E94A2
:101AF000EC1DC82F82E290E00E94EC1D2C2F30E0FC
:101B0000A901582BCA01CF910895CF93C92F682FEF
:101B100084E090E00E94FA1D6C2F82E290E0CF9169
:101B20000C94FA1DAB01BC018FE090E00C940C1EEC
:101B3000AB01BC0183E190E00C940C1E60E070E00E
:101B4000CB010C94980D60E070E0CB010E94920DE7
:101B50000C949E0D69EE7EEF80E090E00E94181ECE
:101B600060E082E090E00E94FA1D60E083E090E097
:101B70000E94FA1D1092DD011092DE011092DF0129
:101B80001092E00160E084E090E00E94FA1D60E0C5
:101B900082E290E00E94FA1D60E085E090E00E9401
:101BA000FA1D60E086E090E00E94FA1D6FEF87E08A
:101BB00090E00E94FA1D40E050E0BA0188E090E019
:101BC0000E940C1E60E08DE090E00E94FA1D40E053
:101BD00050E0BA0188E190E00E940C1E60E087E1CD
:101BE00090E00E94FA1D40E050E0BA018CE190E0E4
:101BF0000E940C1E60E070E080E290E00E94181EDF
:101C000040E050E0BA0188E190E00E940C1E0C9484
:101C1000A30D0C94AA0D682F8EE090E00C94FA1D91
:101C20000E94B116609371027093720280937302E6
:101C30009093740260936D0270936E0280936F02B2
:101C400090937002089585B7806885BF85B78068D6
:101C500085BF089581E008950C942A0E08950C9490
:101C60002E0E0C942E0E0C94310E0C942E0E0C9401
:101C7000350E0C942E0E0E94230E85EE90E10E94EC
:101C8000EF140E94390E0C94370E0E942F0E0C9404
:101C90002E0E0E94FF100C9400030E949C160E94BE
:101CA000F3110E94490E0C94330E5F926F927F9253
:101CB0008F929F92AF92BF92CF92DF92EF92FF925C
:101CC0000F931F93CF93DF93CDB7DEB72A970FB64D
:101CD000F894DEBF0FBECDBF0E940812C82E81113E
:101CE0000E94100E3DE5832E32E0932E00E010E0BE
:101CF000502E802F0E9423115C01F401619071909D
:101D00004F016826792661147104B1F40F5F1F4FEB
:101D10000830110569F78FEF89838A831B820E943F
:101D2000A5168160782F9D838C8349815A816B81B0
:101D30008D810E9420033AC08091750281FD0E942E
:101D40002C11D12CEE24E394F12CC3018E219F2180
:101D5000892B29F10E942C0E8823A9F0DE825F8254
:101D6000AE20BF2081E0AB2809F480E088870E9484
:101D7000A5168160782F9A8789874E815F81688553
:101D80008A850E942003000F111FF801E35AFD4FBE
:101D900080819181E826F926F182E08207C0D39400
:101DA000EE0CFF1CFFE0DF12D0CFB0CF81E0C110FE
:101DB00001C080E02A960FB6F894DEBF0FBECDBFFB
:101DC000DF91CF911F910F91FF90EF90DF90CF9017
:101DD000BF90AF909F908F907F906F905F9008958D
:101DE0000E94550E0C941503CF93DF930E940E10A2
:101DF000EC01811522E59207E8F5811531E593079D
:101E000008F0B6C0883E910528F5803E910508F09F
:101E1000E9C0883A910570F4853A910508F07AC0D6
:101E20008130910509F473C008F4D9C0049708F013
:101E3000D9C0D5C08F3B910508F0D1C0C85AD0E0B9
:101E4000CC0FDD1FCE5BDE4F0990D881C02DCE01B7
:101E50009464C9C0811540E5940708F069C08115F4
:101E600050E4950708F060C09A9581159F4108F4E9
:101E7000B9C0B5C0811536E5930728F5811545E54C
:101E8000940708F092C0811554E5950708F087C0C3
:101E9000AC0143705527282F26952695C115D345AB
:101EA00008F06CC081E090E002C0880F991F4A954D
:101EB000E2F740E2249F90011124EC01C22BD32BC6
:101EC000CE019C6890C081152AE5920780F48115A7
:101ED00039E5930708F072C0811548E5940708F4C6
:101EE0007EC0D82FCC27CE01806F906A7CC09056E0
:101EF0008115904208F073C08D2F8F710E94A2103F
:101F0000DD27D0628F71AE01582BCA016CC081E011
:101F100090E069C0C55AD0E0C059DE4F8881C82F13
:101F2000D0E0CE0190645FC0DF70CE01906A5BC0EC
:101F300074E0969587957A95E1F7282F23703C2FCA
:101F4000337081E090E002C0880F991F3A95E2F764
:101F50009C68AC01522B9A019C2F9F709695969588
:101F600050E2959FE0011124C9018C2B9D2B3BC0B1
:101F7000D82FCC27CE01816F906A35C081E090E0E8
:101F800002C0880F991F4A95E2F750E2259F900101
:101F90001124EC01C22BD32BCE019A6824C0D82F78
:101FA000CC27CE01846F906A1EC00E94A2108F7150
:101FB00090E0D82FCC27CE01906215C08F700E9480
:101FC000A21094E0D695C7959A95E1F7CF70D0E02E
:101FD000DC2FCC27D0699E01282BC90104C080E0EA
:101FE00090E001C0CE01DF91CF91089528E7829F54
:101FF000C0011124FC012FE0729FE00DF11D11249E
:10200000E60FF11DEE0FFF1FE852FF4F85919491EF
:1020100008950E94F60F0E94F40E089582389105EB
:1020200069F1B0F48133910509F46DC048F4893247
:10203000910509F463C08A32910509F469C00895D5
:102040008533910509F455C089339105B9F0089598
:10205000833E910569F138F4803E9105B1F0823EEE
:10206000910509F10895863E9105A9F1873E9105F4
:10207000B9F1843E910509F064C023C02091AA0201
:1020800020FD4FC021FD4DC008958091AA0280FD22
:1020900044C08091AB0280FF44C08091AA0284FDBD
:1020A00042C083EE4DC08091AA0282FF38C0F5CFB6
:1020B0008091AA0282FD33C08091AB0280FD31C0C5
:1020C000ECCF8091AB0281FF32C08091AA0284FDE7
:1020D0002AC087EE35C08091AA0283FF26C0F5CFC3
:1020E0008091AA0283FD21C08091AB0281FD1FC0B7
:1020F000ECCF8091AA0285FD1CC01DC08091AA0270
:1021000085FD19C016C08091AA0286FD16C017C0B1
:102110008091AA0286FD13C010C089E311C082EE2F
:102120000FC080EE0DC080E00BC086EE09C084EECB
:1021300007C089E205C085E303C08AE201C081E3EC
:1021400090E008959091AA0292FF0DC0282F287167
:10215000283019F4877F846006C0282F247124302A
:1021600011F48B7F886093FF0DC0282F28712831D0
:1021700019F4877E846106C0282F2471243111F45C
:102180008B7E88612091AB0220FF0DC0382F387103
:10219000383019F4877F816006C0382F31713130B3
:1021A00011F48E7F886021FF0DC0282F28712831FF
:1021B00019F4877E816106C0282F2171213111F425
:1021C0008E7E886194FD877E089580E008950C944A
:1021D0005B0D0E9408128FE39CE90197F1F700C0A4
:1021E00000000E94081286E00E94231185FF04C0AF
:1021F0000E94E7100C94F21608950C94E9100E94C6
:10220000610D811102C00E94090E0E946C0D809325
:1022100075020E94740D9093AB028093AA020E94F3
:10222000FD100E94700D682F70E080E090E00E9429
:102230007D076091D9017091DA018091DB01909165
:10224000DC010C94B507E82FF0E0EE0FFF1FE4541B
:10225000FD4F808191810895089580EA8A95F1F774
:10226000089500C008950C942D1108950C94351113
:102270000C9436110C9435110C943A11F894E82F03
:10228000E295EF70F0E031A1282F2F7081E090E00F
:1022900001C0880F2A95EAF7982F9095932391A370
:1022A00092A1892B82A3789408950F931F93CF93C3
:1022B000DF93C3E7D1E089918F3F11F00E943E1177
:1022C00081E0C238D807B9F7C2E8D1E00AE811E0E6
:1022D00089918F3F11F00E943E110C171D07C1F725
:1022E000DF91CF911F910F910895AF92BF92DF922E
:1022F000EF92FF920F931F93CF93DF93C62FD0E0FF
:10230000CD58DE4F28812F3F09F463C08A01F62E95
:10231000E92ED82EF894E22FE295EF70F0E091A12B
:10232000822F8F7021E030E001C0220F8A95EAF7FA
:10233000892F822B81A382A12095282322A3789420
:102340000E94311182E8A82E81E0B82EED2DFE2DDD
:102350009F01205F3F4FE12CA80140955095D5018A
:102360006D915D016F3FC9F0862F82958F7090E06F
:10237000DC0190968C9190E06F7002C095958795E6
:102380006A95E2F780FD09C080819181802B912BB5
:1023900091838083EE24E39406C08081918184231D
:1023A0009523918380833296E217F307C1F68881E3
:1023B0008F3F11F00E943E116E2D8F2DDF91CF9136
:1023C0001F910F91FF90EF90DF90BF90AF900C9412
:1023D0003311DF91CF911F910F91FF90EF90DF901C
:1023E000BF90AF9008950E94551180E1ECEBF2E0B0
:1023F000DF01982F1D929A95E9F7ECEAF2E0DF01F0
:102400001D928A95E9F788E00E945D120C947A0289
:10241000CF92DF92FF920F931F93CF93DF93CDB7AD
:10242000DEB760970FB6F894DEBF0FBECDBF8E014A
:102430000F5F1F4F80E1F80111928A95E9F7F12CA7
:10244000CC24C394D12CA6016F2DC8010E94751114
:10245000F394CC0CDD1CFFE0FF12F5CF40E150E01F
:10246000B8018CEA92E00E94DF1DFF24F3940097EC
:1024700009F4F12C892B41F080E1F801ACEAB2E0DB
:1024800001900D928A95E1F72F2D48E06CEB72E0F8
:102490008CEA92E00E945E120E947C028F2D609670
:1024A0000FB6F894DEBF0FBECDBFDF91CF911F9165
:1024B0000F91FF90DF90CF9008950895FF920F93B2
:1024C0001F93CF93DF93F82E092F162FD72FC42FEA
:1024D000222349F081E0809378020E94A516909310
:1024E000770280937602809178028823D9F08091D8
:1024F0007602909177020E94BD16059798F0EF2D15
:10250000F02FA12FBD2F80E090E04C2F50E08417DA
:10251000950734F4219131912D933D930196F7CF96
:1025200010927802DF91CF911F910F91FF90089543
:102530000E949F180E944D0E0C94AB180E94AF1879
:102540000E94F00E0C94C9180E9443160E9486182F
:102550000E943B0E0E9498120E949E120E94450EFD
:10256000FBCFCF93DF93EC01FB018281882309F439
:102570003CC1C430FDE5DF0760F4CB3F9CE5D907E3
:1025800088F49E0122503C452431310508F02EC1CB
:1025900009C0C236EDE5DE0729F0C63AFDE5DF07E2
:1025A00009F024C10E94740D9093AB028093AA029B
:1025B000C1318CE5D80709F4C6C008F042C0C93063
:1025C000ECE5DE0709F49BC000F5C5308CE5D807C3
:1025D00009F485C078F4C330ECE5DE0709F478C06F
:1025E00008F07AC0C230DC4509F0F5C08091AA023B
:1025F0008160EFC0C7309CE5D90709F478C008F0C6
:102600007AC08091AA028061E4C0CD30FCE5DF078A
:1026100009F487C058F4CB309CE5D90709F479C098
:1026200008F07BC08091AA0288606FC0CF30FCE5C3
:10263000DF0709F480C008F082C08091AA02877F7A
:10264000C8C0CE3F9CE5D90709F471C000F5C5317B
:10265000FCE5DF0709F485C068F4C3319CE5D907C0
:1026600009F475C008F095C00E9425078091AA0260
:102670008F77AFC0CC3FFCE5DF07A9F108F054C06D
:10268000CB3FDC4509F0A7C08091AB0240C0C2300F
:10269000EDE5DE0709F489C058F4C1158DE5D807CA
:1026A00009F45AC008F069C08091AB0282602FC063
:1026B000C236EDE5DE0709F47CC0C63AFDE5DF076A
:1026C00009F481C0C330DD4509F085C080E06EC0EB
:1026D0008091AA0282607DC08091AA0216C080917A
:1026E000AA02886076C08091AB0282604FC0809160
:1026F000AA0280626EC08091AA0280646AC00E94B1
:1027000025078091AA02806864C0846062C08160ED
:102710003DC08091AA028E7F5CC08091AA028D7F0D
:1027200058C08091AA0216C08091AB0218C0809157
:10273000AB028D7F2BC08091AA028F7E4AC0809110
:10274000AA028F7D46C08091AA028F7B42C08091F1
:10275000AA02877F8B7F3DC08091AB028D7F8E7FE9
:1027600015C08091AA0282FB222720F991E09227CE
:1027700090FB82F990FB83F92CC08091AB02982FDB
:10278000909591708E7F892B90FB81F98093AB029D
:1027900022C00E9425078091AA0287FB222720F9E8
:1027A00091E0922790FB87F914C081E00E940B0E04
:1027B00012C08091AA0284FB222720F991E092277F
:1027C00090FB84F906C08091AA02982F909590FB07
:1027D00080F98093AA028091AA029091AB020E9494
:1027E000850D0E94250780E001C081E0DF91CF9137
:1027F0000895CF93DF9386319C4541F5EB010E940C
:10280000780C982F8A81209102013091030188234E
:1028100079F09A7A81E009F480E08093790291114D
:1028200002C069E201C065E3C9010E94E1150AC066
:1028300080917902811102C069E201C065E3C9019A
:102840000E94EC150E94BA0C80E001C081E0DF918B
:10285000CF9108950F931F93CF93DF93C42FD22F5F
:10286000FC0182818823C9F040937C020E94A51656
:1028700090937B0280937A0280E28C0F883008F07C
:1028800057C0C77081E001C0880FCA95EAF7DF9191
:10289000CF911F910F910C94910480917C02481369
:1028A00030C080917A0290917B020E94BD16883CD4
:1028B000910538F510E21D0FCD17B9F080E28C0FAD
:1028C000883040F4C77081E001C0880FCA95EAF7EC
:1028D0000E949804183028F581E09D2F977001C060
:1028E000880F9A95EAF70E949104802F0E9488042D
:1028F0001830F0F4D77081E001C0880FDA95EAF75C
:102900000AC080E28C0F883098F4C77081E001C063
:10291000880FCA95EAF7DF91CF911F910F910C9420
:102920009804802FDF91CF911F910F910C94880410
:10293000DF91CF911F910F9108950F939C01CB01CF
:10294000243F4CE5340731F188F4293DFCE53F078D
:10295000D9F02A3D4CE5340779F1283D3C45A9F5ED
:1029600006E221EE41EE68ED7CE52BC0263FFCE55A
:102970003F07E1F0A8F0273F3C4539F507E225EE97
:1029800046EE67EF7CE51DC007E225EE45EE69EDFA
:102990007CE517C006E221EE40EE64EF7CE511C055
:1029A00007E225EE44EE65EF7CE50BC006E221EE82
:1029B00042EE66EF7CE505C008E221E045EE6AEDF7
:1029C0007CE50E942A1480E008C0FC0182818823F3
:1029D00019F010927C0201C081E00F91089590934C
:1029E0008B0180938A0108959093820280938102E3
:1029F0000895E0918102F0918202309721F00190D8
:102A0000F081E02D099480E00895E0918102F09139
:102A10008202309799F020911001222359F02091E1
:102A2000AA0227FF07C0DC012C9111962C93119765
:102A300026E02C930280F381E02D099408952091E3
:102A40007F02309180022817390771F0909380023D
:102A500080937F02E0918102F0918202309721F011
:102A60000680F781E02D0994089520917D02309130
:102A70007E022817390771F090937E0280937D02C1
:102A8000E0918102F0918202309721F00084F1857B
:102A9000E02D09940895FC0132968091100188235D
:102AA00031F08091AA0287FF02C09EE101C096E04A
:102AB00080E0915028F021912223D9F38F5FF9CF44
:102AC0000895662351F1209110012223E9F020910D
:102AD000AA0227FF19C0462F4695469546954E31C6
:102AE000E0F4677021E030E002C0220F331F6A95E6
:102AF000E2F7FC01E40FF11D828190E028233923E5
:102B000081E0232B69F409C0FC01329608962191DB
:102B1000621729F0E817F907D1F780E0089581E0FE
:102B200008959C01FC0132969FEF80E04191461789
:102B300089F09F3F19F4411101C0982F8F5F8630B3
:102B4000A9F79F3F39F0F901E90FF11D97FDFA95BB
:102B50006283089508959C012A5F3F4FFC014281E2
:102B6000461301C01282019682179307B9F70895A0
:102B7000262F2695269526952E3168F4FC01E20F26
:102B8000F11D677021E030E001C0220F6A95EAF77D
:102B90008281282B22830895262F26952695269517
:102BA0002E3170F4FC01E20FF11D677021E030E07E
:102BB00001C0220F6A95EAF720958281282322839B
:102BC000089520911001222329F02091AA0227FDC7
:102BD0000C94B8150C94911520911001222329F022
:102BE0002091AA0227FD0C94CC150C94AB152091D2
:102BF0001001FC013296222331F08091AA0287FF56
:102C000002C08EE101C086E0DF011D928A95E9F7DE
:102C1000089508950C94091683E0809383020C9420
:102C20000A16811102C081E001C082E08093830214
:102C30000C940A160C94111681E0809383020C9474
:102C40000A160C941C1608950C9423160C94241642
:102C50000C9423160C9423160C942316CF930E94E5
:102C60002A160E9408120E942816C0E08C2F0E948B
:102C70002311892B29F4CF5FC830C1F780E001C050
:102C800081E0CF91089508951F920F920FB60F9291
:102C900011248F939F93AF93BF93809184028111EE
:102CA00013C08091CC029091CD02A091CE02B09140
:102CB000CF024196A11DB11D8093CC029093CD020D
:102CC000A093CE02B093CF02BF91AF919F918F910D
:102CD0000F900FBE0F901F9018958091D4028430F2
:102CE00031F10E94E0021092840220E488E190E039
:102CF0000FB6F894A895809360000FBE20936000F3
:102D000083B7817F846083BF83B7816083BF7894FA
:102D1000889583B78E7F83BF0FB6F894A89580916E
:102D20006000886180936000109260000FBE08957B
:102D30000E9425070C94E40282E084BD93E095BDD7
:102D40009AEF97BD80936E0008952FB7F894809105
:102D5000CC029091CD02A091CE02B091CF022FBFB4
:102D600008952FB7F8946091CC027091CD028091B4
:102D7000CE029091CF022FBF08959C014FB7F894D7
:102D80008091CC029091CD02A091CE02B091CF0261
:102D90004FBF821B930B089578941F920F920FB62A
:102DA0000F9211248F939F93AF93BF938091CC0286
:102DB0009091CD02A091CE02B091CF020196A11DBB
:102DC000B11D8093CC029093CD02A093CE02B0931C
:102DD000CF02BF91AF919F918F910F900FBE0F9037
:102DE0001F90189581E08093E00080E28093D800E6
:102DF0001092C9008FE19EE40197F1F700C0000036
:102E000087E090EBDC018093DD029093DE02A093DB
:102E1000DF02B093E0029CE088E10FB6F894A89539
:102E2000809360000FBE90936000FFCF8091A80256
:102E300008950895CF93DF9320911001222339F054
:102E40002091AA0227FF03C060E222E002C068E0EE
:102E500021E02093E9002FEF3091E800215035FD6B
:102E600006C035ED3A95F1F700002111F5CF20911C
:102E7000E80025FF1DC0EC0180911001811105C003
:102E800040E050E068E070E003C070E040E050E0F7
:102E9000CE010E943B198091E8008E778093E80074
:102EA00080E2FE01A8E8B2E001900D928A95E1F778
:102EB000DF91CF910895809385027093870260938C
:102EC00086028091D402843001F582E08093E9008B
:102ED0008FEF9091E800815095FD06C095ED9A9591
:102EE000F1F700008111F5CF8091E80085FF0DC05A
:102EF00040E050E063E070E085E892E00E943B191A
:102F00008091E8008E778093E8000895BC0184E00A
:102F10000C945B17BC0183E00C945B1708958091BF
:102F2000D302811109C00E94CC1A0E94291B8091F2
:102F3000E20084608093E20008951092D302089525
:102F40000C9421166091D00281E0611101C080E0F3
:102F50000C940C169091D40281E0943009F080E03A
:102F60006091D0020C94111642E061EC81E00E9465
:102F7000451A42E261EC82E00E94451A9091D40227
:102F800081E0943009F080E06091D0020C941A1630
:102F90008091D602833009F461C030F4813071F041
:102FA000823009F49AC008958A3009F486C08B30C3
:102FB00009F46CC0893009F0A8C020C08091D50206
:102FC000813A09F0A2C08091E800877F8093E800F1
:102FD0008091D9029091DA02892B21F460E288E88D
:102FE00092E003C060E080E090E070E00E9486190B
:102FF0008091E8008B778093E80008958091D50256
:10300000813209F082C08091D9029091DA02029750
:1030100008F07BC08091E800877F8093E800809172
:10302000E80082FD05C08091D4028111F8CF6DC007
:103030002091F3008091F20090E0922B029731F4FE
:103040008091F100813011F0863021F48091F100FF
:103050008093A8028091E8008B7753C08091D502BD
:10306000813A09F052C08091D9029091DA02892BFD
:1030700009F04BC08091E800877F8093E800809141
:10308000E80080FFFCCF8091100136C08091D5020E
:103090008132D9F58091D9029091DA02892BA9F574
:1030A0008091E800877F8093E8000E947A1A8091DF
:1030B000D702809310010C9425078091D5028132AC
:1030C00021F58091E800877F8093E8000E947A1ABA
:1030D0008091D8028093A90208958091D502813A07
:1030E000A1F48091E800877F8093E8008091E80058
:1030F00080FFFCCF8091A9028093F1008091E800CD
:103100008E778093E8000C947A1A089584B7877FAD
:1031100084BF0FB6F894A895809160008861809371
:103120006000109260000FBE90E080E80FB6F89447
:1031300080936100909361000FBE0C941C160E9456
:10314000CC1A0E94291BE2EEF0E08081846080832B
:1031500078940C94BE1D84E091E00C94F41480915A
:10316000D4028530A9F48091D402853079F40E948C
:103170006D168091D2028823B1F30E942E16882307
:1031800091F30E9425190E942507EDCF0C94981603
:10319000089508950C94CC18292F33272330310536
:1031A000C9F060F42130310581F02230310509F099
:1031B00044C08BE390E022EE32E043C0213231057F
:1031C000E1F02232310549F138C082E190E02DE191
:1031D00033E037C099278130910549F028F00297F4
:1031E00061F5E8EBF2E005C0EEEDF2E002C0EEECD6
:1031F000F2E0849190E09F0124C06115710541F0D7
:1032000061307105D1F489E090E02DE033E019C020
:1032100089E090E024EF32E014C06115710541F0BF
:103220006130710551F48DE690E02FE233E009C082
:1032300080E490E02CE933E004C080E090E020E0FE
:1032400030E0FA0131832083089580E189BD82E175
:1032500089BD09B400FEFDCF8091D8008F7D809399
:10326000D8008091E00082608093E0008091E000CF
:1032700081FDFCCF0895CF92DF92EF92FF920F93E2
:103280001F93CF93DF93EC018B017A010E94991A6F
:10329000811133C0E114F10439F0F701808191818B
:1032A000081B190BC80FD91FC12CD12C01151105F2
:1032B00019F18091E80085FD16C08091E8008E77B5
:1032C0008093E800E114F10449F0F70180819181D5
:1032D000C80ED91ED182C08285E00FC00E94991A03
:1032E000882321F30AC089918093F10001501109CC
:1032F000FFEFCF1ADF0ADACF80E0DF91CF911F9185
:103300000F91FF90EF90DF90CF9008952091DB0216
:103310003091DC022617370748F06115710539F442
:103320002091E8002E772093E80001C0B901FC014C
:1033300020E06115710579F18091D4028823F1F1C3
:103340008530F1F18091E80083FD3CC08091E80078
:1033500082FD2EC08091E80080FFEBCF2091F3002A
:103360008091F20090E0922B6115710551F0883048
:10337000910538F421912093F10061507109019673
:10338000F3CF21E0089709F020E08091E8008E77E4
:103390008093E800CECF2111CFCF0AC08091D40214
:1033A000882361F0853061F08091E80083FD0AC0D8
:1033B0008091E80082FFF2CF80E0089582E00895D6
:1033C00083E0089581E008952091DB023091DC02D2
:1033D0002617370748F06115710539F42091E80088
:1033E0002E772093E80001C0B901FC0120E06115AF
:1033F000710591F18091D402882309F440C0853091
:1034000009F43FC08091E80083FD3DC08091E80051
:1034100082FD2FC08091E80080FFE9CF2091F3006A
:103420008091F20090E0922B6115710559F088307F
:10343000910540F424912093F10031966150710977
:103440000196F2CF21E0089709F020E08091E80092
:103450008E778093E800CBCF2111CCCF0AC080912A
:10346000D402882361F0853061F08091E80083FD0B
:103470000AC08091E80082FFF2CF80E0089582E0E8
:10348000089583E0089581E00895982F973068F5B6
:103490009093E900981739F07091EC002091ED00BD
:1034A0005091F00003C0242F762F50E021FD02C080
:1034B0009F5FECCF3091EB003E7F3093EB0030917B
:1034C000ED003D7F3093ED003091EB0031603093A3
:1034D000EB007093EC002093ED005093F0002091EE
:1034E000EE0027FDE5CF80E008958F708093E9001E
:1034F00081E008958091D50287FF11C08091E80096
:1035000082FD05C08091D4028111F8CF11C0809155
:10351000E8008B770BC08091D402882349F080911A
:10352000E80080FFF8CF8091E8008E778093E80074
:1035300008952091E4003091E50095E64091EC007B
:10354000842F817040FF23C08091E80080FD1DC062
:103550008091D402882399F0853099F08091EB0016
:1035600085FD11C04091E4005091E5002417350716
:1035700029F3915011F09A01E1CF84E0089582E09F
:10358000089583E0089581E0089580E008954091D2
:10359000E80042FFDDCF08950E943A1B0E94421BC3
:1035A000E0EEF0E0808181608083E8EDF0E08081F2
:1035B0008F77808319BCA7EDB0E08C918E7F8C93C0
:1035C00080818F7E80831092D30208950F931F9382
:1035D000CF93DF930E943A1B0E94421BC8EDD0E0BC
:1035E00088818F77888388818068888388818F7DB0
:1035F000888319BC1092D4021092D0021092D20289
:103600001092D10200EE10E0F80180818B7F808360
:1036100088818160888342E060E080E00E94451AF2
:10362000E1EEF0E080818E7F8083E2EEF0E0808149
:1036300081608083808188608083F80180818E7FB3
:103640008083888180618883DF91CF911F910F9162
:103650000895E8EDF0E080818F7E8083E7EDF0E073
:1036600080818160808384E082BF81E08093D30287
:103670000C94E61AE8EDF0E080818E7F8083109252
:10368000E20008951092DA001092E10008951F926E
:103690000F920FB60F9211242F933F934F935F9386
:1036A0006F937F938F939F93AF93BF93EF93FF930A
:1036B0008091E10082FF0BC08091E20082FF07C091
:1036C0008091E1008B7F8093E1000E94BD1D80917D
:1036D000DA0080FF1FC08091D80080FF1BC080915E
:1036E000DA008E7F8093DA008091D90080FF0DC0D0
:1036F00080E189BD82E189BD09B400FEFDCF81E092
:103700008093D4020E948F1705C019BC1092D40276
:103710000E949D178091E10080FF19C08091E20016
:1037200080FF15C08091E2008E7F8093E20080913F
:10373000E20080618093E2008091D80080628093F3
:10374000D80019BC85E08093D4020E94A217809112
:10375000E10084FF30C08091E20084FF2CC080E152
:1037600089BD82E189BD09B400FEFDCF8091D800FA
:103770008F7D8093D8008091E1008F7E8093E1005F
:103780008091E2008F7E8093E2008091E200816070
:103790008093E2008091D002882311F084E007C07A
:1037A0008091E30087FD02C081E001C083E0809347
:1037B000D4020E94AA178091E10083FF29C0809162
:1037C000E20083FF25C08091E100877F8093E100C4
:1037D00082E08093D4021092D0028091E1008E7F2B
:1037E0008093E1008091E2008E7F8093E2008091DF
:1037F000E20080618093E20042E060E080E00E94AD
:10380000451A8091F00088608093F0000E94A01714
:10381000FF91EF91BF91AF919F918F917F916F91A8
:103820005F914F913F912F910F900FBE0F901F907E
:1038300018951F920F920FB60F9211242F933F935A
:103840004F935F936F937F938F939F93AF93BF93A8
:10385000CF93DF93EF93FF93C091E900CF708091F6
:10386000EC00D82FD17080FDD0E81092E900809153
:10387000F000877F8093F00078940E945D1C109286
:10388000E9008091F00088608093F000CD2BCF702C
:10389000C093E900FF91EF91DF91CF91BF91AF917C
:1038A0009F918F917F916F915F914F913F912F9158
:1038B0000F900FBE0F901F9018951F93CF93DF931B
:1038C000CDB7DEB7AA970FB6F894DEBF0FBECDBF57
:1038D000E5EDF2E08091F100819322E0ED3DF20709
:1038E000C9F70E94C8178091E80083FF2EC180911C
:1038F000D5029091D602492F50E04A30510508F088
:1039000024C1FA01EE59FF4F0C94D91D803821F0E3
:10391000823809F01AC108C08091D1029091D20278
:10392000992389F082600FC08091D9028F7087300F
:1039300008F00BC18093E9008091EB0085FB88279C
:1039400080F91092E9009091E800977F9093E80049
:103950008093F1001092F100D1C0282F2D7F09F043
:10396000F4C0882319F0823061F0EFC08091D70253
:10397000813009F0EAC0933009F080E08093D202F0
:103980002EC08091D70281112AC08091D9028F70F8
:103990002FEF280F263008F0D8C08093E90020913F
:1039A000EB0020FF1CC0933021F48091EB0080627B
:1039B00014C09091EB0090619093EB0021E030E017
:1039C000A90102C0440F551F8A95E2F74093EA000F
:1039D0001092EA008091EB0088608093EB001092D7
:1039E000E9008091E800877F8093E8000E947A1ABE
:1039F000ACC08111AAC01091D7021F778091E3005B
:103A00008078812B8093E3008091E800877F80930A
:103A1000E8000E947A1A8091E80080FFFCCF809134
:103A2000E30080688093E300111102C082E001C0CE
:103A300083E08093D40289C08058823008F085C02A
:103A40008091D7029091D8028C3D53E0950779F58B
:103A500083E08A838AE289834FB7F894DE01139664
:103A600020E03EE051E2E32FF0E050935700E49174
:103A700020FF03C0E295EF703F5FEF708E2F90E064
:103A8000EA3010F0C79601C0C0968D939D932F5FCA
:103A9000243149F74FBF8091E800877F8093E80089
:103AA0006AE270E0CE0101960E94861916C060910C
:103AB000D9027091DA02AE014F5F5F4F0E94CA18BF
:103AC000BC01892B09F441C09091E800977F909345
:103AD000E80089819A810E94E4198091E8008B773F
:103AE0008093E80032C0803881F58091E800877FBC
:103AF0008093E8008091D0028093F1008091E800EB
:103B00008E7772CF811121C08091D7029091D80217
:103B100099270297D4F48091E800877F8093E8008A
:103B20008091D7028093D0020E947A1A8091D002AD
:103B3000811106C08091E30087FD02C081E001C0D1
:103B400084E08093D4020E94B4178091E80083FF40
:103B50000AC08091E800877F8093E8008091EB00A5
:103B600080628093EB00AA960FB6F894DEBF0FBE7A
:103B7000CDBFDF91CF911F9108950895CF9380918C
:103B8000D4028823A1F0C091E900CF709091EC009D
:103B9000892F817090FD80E8C82B1092E9008091F8
:103BA000E80083FD0E945D1CCF70C093E900CF91B7
:103BB0000895EE0FFF1F0590F491E02D0994FB018D
:103BC000DC0104C08D910190801921F441505040D6
:103BD000C8F7881B990B0895F999FECF92BD81BD56
:103BE000F89A992780B50895A8E1B0E042E050E046
:103BF0000C94201E262FF999FECF92BD81BDF89A14
:103C0000019700B4021639F01FBA20BD0FB6F89420
:103C1000FA9AF99A0FBE08950396272F0E94FB1D6A
:103C20000E94FA1D252F0E94FB1D242F0C94FB1DC2
:103C30000196272F0E94FB1D0C94FA1DDC01CB017D
:103C4000FC01F999FECF06C0F2BDE1BDF89A3196AC
:103C500000B40D9241505040B8F70895F894FFCF4A
:103C6000C8003B0216171A178E178A1786171917DE
:103C700001E200E900EA00B500B600B700CD00831C
:103C800001CC008A01920194012102230224022521
:103C900002260227022A02B300B4006F00700081DE
:103CA0008283E200E900EA00B500B600B700CD006B
:103CB0008301CC008A019201940121022302240293
:103CC0002502260227022A02B300B4006F0070000A
:103CD00081828333F1319592919094969734353661
:0A3CE000666793F5F4F03732C63042
:00000001FF
